:020000020000FC
:100000000CC04FC00000000076C079C080C0000066
:1000100000000000626B6F3330320FED0DBF00E067
:1000200008BB0CEF07BB08E702BB00E001BB02E026
:1000300003BF02E00EBD77278827DAD104E6B02E91
:10004000CAD0C9D0B3D004E6302E06EF202E00E08F
:10005000C02ED02E02EC08BF09BF789400E00093B8
:100060006A0000936B0000936C0000936D0003E046
:1000700005BF00E40BBF2AE083FFFECF092D1A2D38
:10008000877F0C541440B8F72A95B1F7F8948ED0B6
:100090008DD07894F9E07F7D7061B4D09DD159D135
:1000A000B3C11FB644274BBF45B740FF09C0829B71
:1000B0001EC042E045BF4CB55DB5742E852E17C0FD
:1000C000829915C043E045BF83FD11C04CB55DB5B5
:1000D00047195809942EA52E483968E0560738F478
:1000E000403263E0560718F0886044E6B42E50E4CE
:1000F0005BBF1FBE18951FB67E7F1FBE18951FB62B
:1001000043949160BB2009F0BA941FBE18951FB6A6
:1001100076FD28C0422D562D541730F43A9459F4E8
:1001200054E6352E4A9506C031F03A9421F450E554
:10013000352E4395242E706474FF08C077FF03C0EA
:10014000839B72607F7781FFC79807C075FF03C0EC
:1001500081FFC59802C081FFC698422D4C59409539
:1001600042BF22C0422D42BF7F7B74FF03C080FF8D
:10017000C79A07C075FF03C080FFC59A02C080FF01
:10018000C69A4D3918F482608E7F07C0463F18F03A
:100190008D7F816002C08D7F8E7F87FF05C0C69BEB
:1001A00003C0459B74608F771FBE18958B9A10E82B
:1001B000002702BFC29AC69A02B70032E9F7C29876
:1001C000C69828E0002702BF02B70F3FE9F72A953B
:1001D000C9F71A9569F710E828E0002702BF02B7AF
:1001E0000F3FE9F72A95C9F71A95B1F78B9808954B
:1001F00030E03BBF30E03EBD32E00CB51DB5242DF4
:100200003EBD0895F5DF30E43BBF009360001093DE
:10021000610020936200C0916300D0916400E0917E
:1002200065000C1B1D0B2E0B34E0269517950795CA
:100230003A95D9F7C02FD12FE22F222371F41093D2
:100240006E00112321F000501D4738F408C0122D14
:10025000159515951A5C011710F4BED008C0C0930F
:100260006600D0936700C0936800D0936900009146
:100270006000109161002091620000936300109370
:10028000640020936500089530E010E000916D0057
:1002900020916C00020F131F20936D0020916B00C2
:1002A000020F131F20936C0020916A00020F131F8E
:1002B00020936B001695079516950795F02F8F7D67
:1002C000089583FF16C0092D1A2D877F0C54144002
:1002D00010F4002711271695079516950795169582
:1002E0000795202F0456104008F024E620936A005A
:1002F0008062089590FF17C09E7F72FF06C07B7FCB
:100300004C2D433090F4C39403C0CC2009F0CA9420
:1003100071FF06C07D7F4D2D443628F4D39403C071
:10032000DD2009F0DA943FD00895F89476CE71601C
:10033000C0916600D09167005BDFC00FD11F02E85B
:1003400009BFDBBDCABD02EC09BF30E43BBF70FD95
:10035000FECF71604DDFC0E8DBEB0C0F1D1F22E804
:1003600029BF1BBD0ABD22EC29BF30E43BBF089565
:1003700071603EDFC0916800D09169000C0F1D1FB5
:1003800022E829BF1BBD0ABD22EC29BF30E43BBFD8
:1003900082FD38DF85FD78DF84FD93DF86FDAADFEF
:1003A00070FDFECF08950F2F0D1908F409E010918C
:1003B0006E00183038F014E616951695011748F0BF
:1003C000012F07C0143028F014E61695011708F025
:1003D000012F0095602E089506EF202E08E000936F
:1003E0006E00C0E0DDE7C0936600D093670008951B
:1003F00006EF602E00E008BB04E6302E8160089511
:1004000004E00A95F1F7089570FD01C006C0859BD0
:10041000FBCFF6DF859BF8CFABDFC3980000000071
:1004200080FFC29A84DF706870FD02C04ADF09C095
:100430008499FACFE5DF8499F7CF806199DF8F7EC9
:100440007F7700EC09BF7F7D7F7E81FD02C076FD56
:1004500003C0C79880FFC69A02EC09BF68DF70FD31
:1004600003C085FD11DF06C0869BF9CFC9DF869BDF
:10047000F6CF7EDFC2980000000080FFC49A57DFED
:10048000806870FD01C007C08599FBCFB9DF8599F1
:10049000F8CF6EDF8F7700EC09BF70627F7E81FD41
:1004A00002C076FD03C0C69880FFC59A02EC09BF62
:1004B0003EDF70FD02C01EDF08C0849BFACFA0DFC4
:1004C000849BF7CF806454DF8F7BC49800000000CA
:1004D00080FFC39A2CDF70FD02C094DE08C08699AD
:1004E000FACF8EDF8699F7CF846042DF8B7F00ECF6
:1004F00009BF7F7D706181FD02C076FD03C0C59894
:1005000080FFC79A02EC09BF12DFBB2009F07CCF45
:04051000F89483CD0B
:00000001FF
